:0200000480007A
:100000006F00C004732F2034930F8000630AFF0336
:10001000930F90006306FF03930FB0006302FF038A
:10002000170F0080130F0FFE63040F0067000F000F
:10003000732F203463540F006F004000136E9E53E3
:10004000171F00002320CFFD6FF09FFF732540F1A5
:100050006310050073251030635805000F00F00F82
:10006000130E100073000000130E00009702000032
:10007000938282F973905230735020307350303035
:1000800073504030970200809382C2F7638C020065
:10009000739052109302B01A739022307323203061
:1000A000E39E62F873500030970200009382420191
:1000B00073901234732540F17300203097200000B4
:1000C000938040F483D10000930EF00F130E2000B4
:1000D0006396D127972000009380C0F283D120003F
:1000E000B70E0100938E0EF0130E30006398D125E9
:1000F00097200000938000F183D14000B71E0000DC
:10010000938E0EFF130E4000639AD12397200000B8
:10011000938040EF83D16000B7FE0000938EFE0015
:10012000130E5000639CD121972000009380E0EDD6
:1001300083D1A0FF930EF00F130E60006390D121C6
:1001400097200000938060EC83D1C0FFB70E0100C0
:10015000938E0EF0130E70006392D11F9720000053
:100160009380A0EA83D1E0FFB71E0000938E0EFFBC
:10017000130E80006394D11D972000009380E0E867
:1001800083D10000B7FE0000938EFE00130E900096
:100190006396D11B972000009380C0E6938000FEF9
:1001A00083D10002930EF00F130EA0006398D119B3
:1001B00097200000938000E59380B0FF83D170000A
:1001C000B70E0100938E0EF0130EB0006398D11796
:1001D000130EC00013020000972000009380A0E2DD
:1001E00083D1200013830100B71E0000938E0EFF01
:1001F0006316D3151302120093022000E31E52FC73
:10020000130ED00013020000972000009380C0DF7F
:1002100083D120001300000013830100B7FE00000B
:10022000938EFE00631CD311130212009302200070
:10023000E31C52FC130EE0001302000097200000A4
:10024000938040DC83D120001300000013000000E5
:1002500013830100B70E0100938E0EF06310D30FCD
:100260001302120093022000E31A52FC130EF00056
:1002700013020000972000009380E0D883D1200073
:10028000B71E0000938E0EFF639AD10B130212006B
:1002900093022000E31052FE130E0001130200002F
:1002A00097200000938040D61300000083D12000E7
:1002B000B7FE0000938EFE006392D1091302120074
:1002C00093022000E31E52FC130E100113020000E3
:1002D00097200000938000D313000000130000005B
:1002E00083D12000B70E0100938E0EF06398D105E4
:1002F0001302120093022000E31C52FC972100001D
:10030000938141D003D1010013012000930E2000FE
:10031000130E20016314D10397210000938181CE35
:1003200003D101001300000013012000930E2000F0
:10033000130E30016314D101631CC0010F00F00FD4
:1003400063000E00131E1E00136E1E0073000000DB
:100350000F00F00F130E100073000000731000C0A8
:10036000000000000000000000000000000000008D
:10037000000000000000000000000000000000007D
:040380000000000079
:1010000000000000000000000000000000000000E0
:1010100000000000000000000000000000000000D0
:1010200000000000000000000000000000000000C0
:1010300000000000000000000000000000000000B0
:081040000000000000000000A8
:10200000FF0000FFF00F0FF00000000000000000D4
:040000058000200057
:00000001FF
